:100000000C943E000C9448000C9448000C9448005A
:100010000C9448000C9448000C9448000C94480040
:100020000C9448000C9448000C9448000C94480030
:100030000C9448000C9448000C9448000C94480020
:100040000C9448000C9448000C9448000C94480010
:100050000C9448000C9448000C9448000C94480000
:100060000C9448000C9448000C9448000C944800F0
:100070000C9448000C9448000C94480011241FBEB6
:10008000CFEFD0E1DEBFCDBF0E944A000C946100EB
:100090000C940000089A82B182B92FEF84E39CE0AF
:1000A000215080409040E1F700C0000010982FEFF1
:1000B00084E39CE0215080409040E1F700C00000C4
:0600C000EACFF894FFCF27
:00000001FF
